:020000040000FA
:040000000CEF02F00F
:040008000EEF00F007
:0800180040EF00F09EA221EF71
:1000200000F09E929F2B9FB1110000EE80F010EE29
:100030008EF0070E9E6FFF0ED76EFF0ED66ED58E1A
:100040001100E61C8116E61C8216D59EF2949E07CE
:10005000EE1CD76EEE1CD66E9E53D8A4D58E000033
:100060000000000000000000000000000000000090
:10007000000000000000E6508112E55082121100DD
:100080001000A69CA69EA19865C0A8FF64C0A9FF09
:10009000A684550EA76EAA0EA76EA682A1A84EEF43
:1000A00000F0A6941200A69CA69E64C0A9FFA6809C
:1000B000A8CF65F01200080E616F62AF829E62BF2A
:1000C000828E0000818C819C6237612F5DEF00F091
:1000D0001200948E080E616F626BD890623782BEF8
:1000E0006281818C819C612F6EEF00F0949E1200E2
:1000F000819E450E626F5BEC00F069EC00F069ECEC
:1001000000F062C068F069EC00F062C069F069EC70
:1001100000F062C06AF069EC00F062C06BF069EC5C
:1001200000F062C071F069EC00F062C070F069EC40
:1001300000F062C073F069EC00F062C072F069EC2C
:1001400000F062C075F069EC00F062C074F069EC18
:1001500000F062C077F069EC00F062C076F069EC04
:1001600000F062C079F069EC00F062C078F069ECF0
:1001700000F062C07BF069EC00F062C07AF069ECDC
:1001800000F062C07DF069EC00F062C07CF069ECC8
:1001900000F062C07FF069EC00F062C07EF0818EFA
:1001A0001200819E000E626F5BEC00F0000E626F29
:1001B0005BEC00F0818E819E060E626F5BEC00F0BE
:1001C000540E626F5BEC00F0750E626F5BEC00F03A
:1001D000C50E626F5BEC00F02A0E626F5BEC00F004
:1001E000818E060EF76E040EF66EFF0E636F330EF1
:1001F000606F632B0900F528FCE0819E63C062F00C
:100200005BEC00F0F5CF62F05BEC00F0818E602FCC
:10021000F9EF00F0819E020E626F5BEC00F0010EC0
:10022000626F5BEC00F0818E819E020E626F628DC8
:100230005BEC00F0000069EC00F0818E62B114EF1D
:1002400001F0819E240E626F5BEC00F0130E626F72
:100250005BEC00F0818E819E260E626F5BEC00F0FD
:100260003B0E626F5BEC00F0818E819E0F0E626F21
:100270005BEC00F0000E626F5BEC00F0818E819E03
:10028000020E626F5BEC00F0020E626F5BEC00F03E
:10029000818E819E020E626F628D5BEC00F0000029
:1002A00069EC00F0818E62B349EF01F0819E0F0E80
:1002B000626F5BEC00F0A00E626F5BEC00F0818E71
:1002C000819E020E626F5BEC00F0020E626F5BECCF
:1002D00000F0818E819E020E626F628D5BEC00F0F9
:1002E000000069EC00F0818E62B36AEF01F0819E3C
:1002F000250E626F5BEC00F0080E626F5BEC00F0A5
:10030000818E1200676B819EA00E626F5BEC00F025
:10031000818E819EF00E626F5BEC00F0818E819E7B
:100320000F0E626F5BEC00F0000E626F5BEC00F092
:10033000818E819EC00E626F5BEC00F0818EB19069
:10034000270EB36EB31E100EB26EB21EA192B18014
:10035000A1A2A8EF01F067B5829467A5828481A865
:10036000B7EF01F0672F9FEF01F0E6EF01F0819EFC
:10037000000E626F628D5BEC00F0000069EC00F033
:10038000818E62BB83EF01F062BD83EF01F078ECF8
:1003900000F0646B68C065F041EC00F0642B69C04C
:1003A00065F041EC00F0642B6AC065F041EC00F0B0
:1003B000642B6BC065F041EC00F068C06CF069C064
:1003C0006DF06AC06EF06BC06FF01200646B53EC9E
:1003D00000F065C06CF0642B53EC00F065C06DF06C
:1003E000642B53EC00F065C06EF0642B53EC00F00E
:1003F00065C06FF012008C2F08EF02F0100E8C6FAA
:10040000060EF76E380EF66E8D51F626D8B0F72A26
:100410000900F504666F1200D38CD38AD388D3A465
:100420000FEF02F0806A816A826A82849494818EDE
:10043000939E828E949E819C939C939A9492949A7C
:10044000949C949694987E6A7F6A000E8E6F000E3C
:100450008F6F200E906F000E916F000E926F020E44
:10046000936F000E946F200E956F000E966F400EE6
:10047000976F000E986F080E996F000E9A6F100E0E
:100480009B6F000E9C6F000E9D6FD56AD580F29415
:10049000F28AF90ECB6ECA6ACA8CCA86CA829E924A
:1004A0009D829F82F28CF28EB16AB18EB18AA19246
:1004B000DC0E816F836F856F876F896F8B6F050E81
:1004C000806F826F846F866F886F8A6FCA84B190E5
:1004D000270EB36EB31E100EB26EB21EA192B18083
:1004E000A1A270EF02F0D1EC00F0000082EC01F06C
:1004F0006C39F00B8D6F010E8C6FFBEC01F0819E5F
:10050000A00E626F5BEC00F0818E819EF00E626F38
:100510005BEC00F0818E819E0F0E626F5BEC00F051
:1005200066C062F05BEC00F0818E819EC00E626F4F
:100530005BEC00F0818EB190050EB36EB31EDC0E45
:10054000B26EB21EA192B180A1B2FDEF02F081B8ED
:10055000A4EF02F0819E000E626F628D5BEC00F0F2
:10056000000069EC00F0818E62BBA4EF02F062BD76
:10057000A4EF02F078EC00F06C516863A4EF02F095
:100580006D516963A4EF02F06E516A63A4EF02F04B
:100590006F516B63A4EF02F08284F29E70C080F012
:1005A00071C081F0F28E00000000F29E72C082F0F5
:1005B00073C083F0F28E00000000F29E74C084F0DD
:1005C00075C085F0F28E00000000F29E76C086F0C5
:1005D00077C087F0F28E00000000F29E78C088F0AD
:1005E00079C089F0F28E00000000F29E7AC08AF095
:1005F0007BC08BF0F28E7DEF02F08294FBEC01F079
:100600007DEF02F0FF42001400FFFF000000000138
:10061000210500509E4B0002162B120062808000C4
:100620000A32C30F13C300FF00003B0017478003CB
:1006300001451800010FFF000A5A14641E6E287845
:1006400032823C8C469650A0A05096468C3C82321A
:1006500078286E1E64145A0A0A5A50A014644696EA
:100660001E6E3C8C28783282823278288C3C6E1E3A
:1006700096466414A0505A0A28780A5A50A0146466
:100680001E6E3C8C32824696964682328C3C6E1EA2
:100690006414A0505A0A782850A028780A5A1E6E6E
:1006A0003C8C3282469614646414964682328C3CAA
:1006B0006E1E5A0A7828A05050A046963C8C287886
:1006C0000A5A32821E6E146464146E1E82325A0AF2
:1006D00078288C3C9646A05046963C8C50A02878B2
:1006E0000A5A1E6E32821464641482326E1E5A0AD2
:1006F0007828A0508C3C964646960A5A3C8C146446
:1007000050A028781E6E328282326E1E7828A05049
:1007100064148C3C5A0A964646960A5A50A03C8C61
:1007200028781E6E32821464641482326E1E782819
:080730008C3CA0505A0A9646C9
:020000040030CA
:03000100080914D7
:02000500800079
:0600080003C003E0034009
:0200000400F00A
:040000004D434850D4
:00000001FF
